:103800000C94341C0C94511C0C94511C0C94511CA1
:103810000C94511C0C94511C0C94511C0C94511C74
:103820000C94511C0C94511C0C94511C0C94511C64
:103830000C94511C0C94511C0C94511C0C94511C54
:103840000C94511C0C94511C0C94511C0C94511C44
:103850000C94511C0C94511C0C94511C0C94511C34
:103860000C94511C0C94511C11241FBECFEFD4E0BA
:10387000DEBFCDBF11E0A0E0B1E0E6E2FFE302C0B1
:1038800005900D92A230B107D9F712E0A2E0B1E0A5
:1038900001C01D92AD30B107E1F70E94861D0C9466
:1038A000921F0C94001C982F8091C00085FFFCCFC4
:1038B0009093C60008951F93282F992787FD909510
:1038C000807F907095958795959587959595879527
:1038D000959587958A304CF0982F995A822F8F7042
:1038E0008A304CF0182F195A08C0982F905D822FFB
:1038F0008F708A30BCF7182F105D892F0E94531CDF
:10390000812F0E94531C1F910895EF92FF920F93F5
:103910001F93EE24FF2487018091C00087FD17C00C
:103920000894E11CF11C011D111D81EAE81685E2D5
:10393000F80686E2080780E0180770F3E0910401BA
:10394000F091050109958091C00087FFE9CF809132
:10395000C600992787FD90951F910F91FF90EF90DA
:1039600008950F931F930E94851C182F0E94531CCB
:103970000E94851C082F0E94531C11362CF01755ED
:1039800001363CF0075508C01033D4F3105301360C
:10399000CCF700330CF000531295107F100F812FDD
:1039A000992787FD90951F910F910895282F8823BF
:1039B00051F090E08091C00087FFFCCF8091C6005D
:1039C0009F5F2917B9F708951F93182F0E94851C30
:1039D000803269F0809103018F5F8093030185300D
:1039E00079F4E0910401F0910501099509C084E1A1
:1039F0000E94531C812F0E94531C80E10E94531C83
:103A00001F9108950E94851C803271F080910301FE
:103A10008F5F80930301853009F00895E0910401E0
:103A2000F09105010995089584E10E94531C80E1FD
:103A30000E94531C0895CF93DF93CDB7DEB7249730
:103A40000FB6F894DEBF0FBECDBF482F882309F410
:103A50004EC010920A0220E030E02D9A19821A829C
:103A60001B821C8289819A81AB81BC8180529E44D9
:103A7000A040B040A0F489819A81AB81BC810196BD
:103A8000A11DB11D89839A83AB83BC8389819A81EF
:103A9000AB81BC8180529E44A040B04060F32D9821
:103AA00019821A821B821C8289819A81AB81BC8116
:103AB00080529E44A040B040A0F489819A81AB819D
:103AC000BC810196A11DB11D89839A83AB83BC8300
:103AD00089819A81AB81BC8180529E44A040B040D4
:103AE00060F32F5F3F4F241708F4B7CF04C0109244
:103AF0000A0243E0B0CF20930A0224960FB6F8944E
:103B0000DEBF0FBECDBFDF91CF9108950F931F93FE
:103B1000CF93DF93000080E48093C4001092C5002F
:103B200088E18093C10086E08093C2005098589A43
:103B3000259A83E00E941B1D0E94851C8033B1F1F1
:103B40008133B9F1803409F454C0813409F45AC086
:103B5000823409F469C0853409F46CC0803531F1D0
:103B6000813521F1823511F1853509F469C0863539
:103B700009F471C0843609F475C0843709F4D0C0E3
:103B8000853709F424C1863709F44AC080910301BE
:103B90008F5F80930301853079F6E0910401F09105
:103BA000050109950E94851C803351F60E94021D73
:103BB000C3CF0E94851C803249F784E10E94531CC8
:103BC00081E40E94531C86E50E94531C82E50E94FA
:103BD000531C80E20E94531C89E40E94531C83E51D
:103BE0000E94531C80E50E94531C80E10E94531CDC
:103BF000A3CF0E94851C8638C8F20E94851C0E94B3
:103C0000021D9ACF0E94851C803809F4F9C08138C2
:103C100009F4FAC0823809F4FBC0883909F4ECC011
:103C200080E00E94E41C88CF84E10E94D61C0E94A0
:103C3000021D82CF85E00E94D61C0E94021D7CCF0F
:103C40000E94851C809306010E94851C80930701B9
:103C50000E94021D71CF84E00E94D61C80E00E9469
:103C6000E41C6ACF0E94851C809309020E94851C77
:103C70008093080280910C028E7F80930C020E9438
:103C8000851C853409F4C8C080910802909109020E
:103C9000892B89F0C0E0D0E008E011E00E94851C8B
:103CA000F80181938F012196809108029091090279
:103CB000C817D90798F30E94851C803209F066CF97
:103CC00080910C0280FFC0C06091080270910902CF
:103CD00061157105F1F0A0910601B09107019D01F8
:103CE00040E050E0E8E0F1E0F999FECF32BD21BDBF
:103CF000819180BDFA9AF99A4F5F5F4F2F5F3F4FD6
:103D00004617570789F7A60FB71FB0930701A0936F
:103D1000060184E10E94531C80E10E94531C0CCFD9
:103D20000E94851C809309020E94851C80930802D2
:103D30000E94851C853409F475C080910C028E7F29
:103D400080930C028091060190910701880F991FC2
:103D500090930701809306010E94851C803209F030
:103D6000EBCE84E10E94531C20910802309109029D
:103D700021153105E9F1C0E0D0E0E0910601F091B4
:103D800007010BC081FF54C03196F0930701E09307
:103D900006012196C217D30758F580910C0280FFC7
:103DA000F1CFF999FECFF2BDE1BDF89A80B50E943E
:103DB000531CE0910601F09107013196F093070141
:103DC000E09306012091080230910902E2CF0E949F
:103DD000851C803209F0DACE84E10E94531C8EE10A
:103DE0000E94531C84E90E94531C86E00E94531CCD
:103DF00080E10E94531CA0CE83E00E94E41C9CCE74
:103E000082E00E94E41C98CE81E00E94E41C94CEE3
:103E100080E10E94E41C90CE80910C02816080932E
:103E20000C0232CF80910C02816080930C0294CFFF
:103E300084910E94531C2091080230910902E09164
:103E40000601F0910701A0CF8091070187FD66C0B0
:103E500010920B028091060190910701880F991F23
:103E600090930701809306018091080280FF09C0AA
:103E70008091080290910902019690930902809323
:103E80000802F894F999FECF1127E0910601F0910C
:103E90000701C8E0D1E0809108029091090210303A
:103EA00091F40091570001700130D9F303E00093C1
:103EB0005700E8950091570001700130D9F301E1F6
:103EC00000935700E89509901990009157000170F0
:103ED0000130D9F301E000935700E89513951034B1
:103EE00098F011270091570001700130D9F305E0D7
:103EF00000935700E8950091570001700130D9F305
:103F000001E100935700E8953296029709F0C7CF78
:103F1000103011F00296E5CF1124FBCE81E08093A2
:063F20000B0298CFFFCF59
:023F2600800019
:0400000300003800C1
:00000001FF
